:020000040000FA
:0400000000001028C4
:08000800F1000308F2000A08F0
:10001000F30073088A0072088300F10E710E090064
:10002000860183160313811307178717A0308700F3
:100030007F308600FF30850083128A273C308500A0
:10004000B501A601D301DA01DB01DC01DE01EE011D
:10005000B801A701D001A801D101A901AA01AB01F2
:10006000AC01C601D201DF01C501E901ED01CF01FB
:100070000230CB000712F601F7011E30DD001C3004
:10008000E30064306E2708308A00052000308A00C3
:10009000C615D2164F14CF10CF124F11CF114F12D9
:1000A0004F135211CF1952154F1B521546110B10F9
:1000B0008B15FF30F800F9006430FA00D10AD10B3B
:1000C00062285213C61F6A285A08D100DA0150214B
:1000D000C6135E289B20A320C726291870287E28D7
:1000E000CF1C7928A91A7928A9187D2810307E27D5
:1000F0007D2825262608EA25F92549216425C00002
:10010000C01B9828401C8C2849215F10D30AD30BB0
:100110008B285F145E28C513C01C8F28AB28401D98
:100120009228C528C01D5E286508942749245E28AA
:100130004619A3275E285F1C0800C51B0800FD3078
:100140009427C5170800DF1C0800451B0800FD3078
:100150009427451708006508C0000830E9004008EA
:100160000339E907C00DC00D4008F039E907EC017B
:100170008030942769089427670894276808942793
:100180006C089427FF3094275E280830E900E701C7
:10019000E8016708EC00B82825260030EA25F92593
:1001A000C51008002C1864292C196429AC1A64297C
:1001B0002C1B6429CF1DE2284F1E64292808073A0A
:1001C0000319FE28C61D64292808053A03190629C3
:1001D00028080D3A03190B292808153A0319142980
:1001E0002808253A03191D2928081D3A031924292E
:1001F0002808353A03192929280864292F30442171
:1002000064307E27521339304421080014304421D1
:10021000083044210800013044210E3044210430CC
:100220004421323044210800143044210830442154
:10023000053044213230442108000F30442106307B
:10024000442132304421080001304421323044211D
:100250000800143044210F3044213230442108007A
:10026000C613CC006A24C40AC40B3B293230442193
:10027000D101DA01080044084421CC0A2A083B3A9B
:10028000031D43292C163229AA0003307E2752135E
:100290007C2B08308A001B2001308A00291E0800B0
:1002A0005108003A031908005108A800A91E5E2948
:1002B00009308A00B22101308A00080028089327FB
:1002C000C619D2284F1AD228C51E6A297608F70007
:1002D0002808F600CF1D6E294F1E1B2BDA0ADA0BF9
:1002E00072291B2B51085024AA005A085024C70019
:1002F0001F302A02031881291F30470203189D2945
:100300001B2B2A08C4001E30C402B921C41F1B2B9A
:10031000441B96294418EB29C418FE294419112AB4
:10032000C419242A441AD829C41AC5294418372ABA
:10033000C4184A2A44195D2A1B2B4708C4001E30E2
:10034000C402B921C41F1B2B441BB2294418962A8E
:10035000C418A92A4419BC2AC419CF2A441A832ACA
:10036000C41A702A4418E22AC418F52A4419082B22
:100370001B2B0030C40710300318013E8A004408CC
:100380000020C40001308A0008000130C200233080
:10039000C70710300318013E8A0047082320C40015
:1003A00001308A00C40AC40BD6297A2B44083029AC
:1003B0000130C2007B30C70710300318013E8A00AD
:1003C00047087B20C40001308A00C40AC40BE92915
:1003D0007A2B440830290130C200D330C7071030CF
:1003E0000318013E8A004708D320C40001308A0068
:1003F000C40AC40BFC297A2B440830290230C200FD
:100400002B30C70711300318013E8A0047082B2103
:10041000C40001308A00C40AC40B0F2A7A2B440896
:1004200030290230C200DB30C70711300318013E0B
:100430008A004708DB21C40002308A00C40AC40BCA
:10044000222A7A2B440830290230C2008330C707A1
:1004500011300318013E8A0047088321C40002308E
:100460008A00C40AC40B352A7A2B44083029043088
:10047000C2003330C70712300318013E8A00470814
:100480003322C40002308A00C40AC40B482A7A2BE3
:10049000440830290430C2008B30C70712300318DB
:1004A000013E8A0047088B22C40002308A00C40A39
:1004B000C40B5B2A7A2B440830290430C200E33095
:1004C000C70712300318013E8A004708E322C40020
:1004D00002308A00C40AC40B6E2A7A2B44083029E1
:1004E0000130C2004F30AA0710300318013E8A00C5
:1004F0002A084F20C40002308A00C40AC40B812A93
:100500007A2B440830290130C200A730AA071030E6
:100510000318013E8A002A08A720C40002308A007E
:10052000C40AC40B942A7A2B440830290130C20033
:10053000FF30AA0710300318013E8A002A08FF2066
:10054000C40002308A00C40AC40BA72A7A2B4408CC
:1005500030290230C2005730AA0711300318013E7B
:100560008A002A085721C40002308A00C40AC40B3A
:10057000BA2A7A2B440830290230C2000730AA0771
:1005800012300318013E8A002A080722C4000230F4
:100590008A00C40AC40BCD2A7A2B440830290230C1
:1005A000C200AF30AA0711300318013E8A002A08A2
:1005B000AF21C40002308A00C40AC40BE02A7A2B9F
:1005C000440830290430C2005F30AA0712300318F3
:1005D000013E8A002A085F22C40002308A00C40A51
:1005E000C40BF32A7A2B440830290430C200B730F8
:1005F000AA0712300318013E8A002A08B722C40055
:1006000002308A00C40AC40B062B7A2B4408302916
:100610000430C2000F30AA0713300318013E8A00CD
:100620002A080F23C40003308A00C40AC40B192B04
:100630007A2B4408302928083F3A0319D62C280879
:100640002D3A0319EF2C2808123A0319072D280810
:100650002F3A0319232D2808373A0319312D28087A
:100660003B3A031D7A2B4F12CF195215C51E7A2B18
:100670007708043A031D432B4F14CF10CF124F11AC
:10068000CF114F13792B77081A3A031D4E2B4F10B9
:10069000CF14CF124F15CF114F13792B7708323A61
:1006A000031D592B4F10CF14CF124F11CF154F13DD
:1006B000792B7708183A031D642B4F10CF14CF16EF
:1006C0004F11CF114F13792B77080E3A031D6F2B63
:1006D0004F10CF14CF124F11CF114F17792B77082E
:1006E000163A031D792B4F10CF14CF124F15CF118F
:1006F0004F13C5124F24AA00AB01521F882B1F3085
:100700002A02031C882B2A08323A0319882B080076
:1007100052172C1C982B3F30AB002C1DA52B003002
:10072000AB001F302A02031CA52B7E30AB00A52B8B
:100730002C1D9D2B7E30AB00A52B1F302A020318E9
:10074000A52B2C1EA52BBD30AB002A08AB075E24C1
:100750002D085219803E94274924CF18B62B451EE8
:100760003B25451208004516AD00A82B4F19E92B73
:10077000CF19D32BCF1AC22B4F1BF52B451E3B2570
:100780004512080025262D08C0000830F500ED258B
:100790000330C0000330F500ED2507307E27451EED
:1007A0003B25451208004F1AD92B52102D08A024C2
:1007B000E22B52142D0892241F302D020318E22B35
:1007C0002C1AEF120230CB000D24451E3B2545129A
:1007D00008003C30A726F030A7262D08A7260330B6
:1007E0007E27451E3B25451208002D08AE246F08C4
:1007F000FF3A0319072C6F08BB240030BF000330F9
:1008000058260E307E270330BF006F0858260E3062
:100810007E27451E3B25451208006F08FF3A031945
:100820003D2C2D08323A031D1A2C4F1E302C20303F
:10083000EF00302C2D08C0002A3040020318212C74
:10084000302C2D08C000403040020318292C5210D3
:10085000302C2D08C0006A30400203185210302C92
:10086000A918362C32307E2718307E2709266F08CB
:10087000B825C725CB0B342CCB0A28080E3A031910
:100880004F1628081F3A03194F1252154F1A5211CA
:100890000800FF30F800F9006430FA00080028086A
:1008A000C4000030C40718300318013E8A00440811
:1008B0000020C40004308A00440808000030AB0760
:1008C00019300318013E8A002B080021AD000430C6
:1008D0008A000800C2187A2C4219862C0030CC07F6
:1008E0001C300318013E8A004C080024C400043068
:1008F0008A0008000030CC071D300318013E8A0032
:100900004C080025C40004308A0008000030CC07E1
:100910001E300318013E8A004C080026C400043033
:100920008A0008002D08C0000030C0071A300318E4
:10093000013E8A0040080022EF0004308A000800CF
:100940002D08C0008130C0071A300318013E8A000C
:1009500040088122EF0004308A000800C000003007
:10096000C0071B300318013E8A0040080023EF0037
:1009700004308A000800C0004230C0071830031855
:10098000013E8A0040084220EF0004308A0008003F
:100990002C1808002C190800AC1A0800AC132C13F2
:1009A000C61DD42CC6110800C61508003D30B3235F
:1009B000A9122C1BC82C2C1EE52CAC19E52C2C12D2
:1009C000AC13BB30B323A91608002C1CE92C2C1047
:1009D00008002C1408007930B3233B2508007E3032
:1009E000B3232C1B032D2C1EF82CAC19F82CEB2C4C
:1009F0002C1DFF2CAC1C012D2C11AC1008002C154B
:100A00000800AC1408007A30B3233B250800AC1969
:100A10001A2DAC1B142D2C1E1F2D2C16AC15BB3003
:100A2000B3237730B3230800AC132C12AC11BB30C6
:100A3000B32308002C12AC11F730B32308002C1696
:100A40003B30B3230800AC1E292DAC12BE30B323BB
:100A500008002C19C516CF19C516AC163E30B323A5
:100A600008002C1F372D2C13BF30B32308002C1780
:100A70003F30B3230800AC1E402DAC12BE30B32370
:100A80002C1F452D2C13BF30B323AC184A2D2C1D21
:100A90004A2D2C11AC1908002C1E08002A302A02FD
:100AA000031C602D2A08353C031C602D32302A06B9
:100AB0000319602D2E302A060319602DAC1708008B
:100AC0002C12BB30B3230800061BB62DEB26003AD0
:100AD000031DB62DE5011727003A031DB62D40086A
:100AE000E500E601E701E8012627003A031DB62DDF
:100AF0004008E600631266081C396306031D862D54
:100B000066186517E618E517631608346316660855
:100B10001C396306031DB62DE61C912D6508D30014
:100B2000013437274518B62D37274518B62D803A9A
:100B30000319AB2DFD26003A031DB62D4008E70032
:100B4000FD26003A031DB62D4008E8005C27003A58
:100B5000031DB62D0234FD26003A031DB62D4008B4
:100B6000E7005C27003A031DB62D043480342808C2
:100B7000C0000730F500401CC22D2A26C00CF50B22
:100B8000BB2D08001326C00CF50BBB2D0800521C12
:100B9000D42D0530F5001A30C000D8250830F500F6
:100BA0006130C000D82508000530F5000F30C000C6
:100BB000401CDF2D0E26C00CF50BD82D0800132687
:100BC000C00CF50BD82D0800C0000830F500ED254D
:100BD00008002808C0000630F500401CF42D2A2625
:100BE000C00CF50BED2D08002F26C00CF50BED2DDC
:100BF00008001E30C0000530F500401C042E2A26D7
:100C0000C00CF50BFD2D08002F26C00CF50BFD2D9B
:100C1000080007104A265730F4001C2E07104A26F9
:100C20003030F4001C2E07104A2601307A27182E87
:100C300000001930F4001C2E071402307A27071028
:100C400001307A27F40B1C2E0800071042264E3084
:100C5000F400372E071042262B30F400372E0710F1
:100C6000422601307A27342E1630F400372E07142E
:100C700002307A270000071001307A273F2EF40B4C
:100C8000372E080031307A2731307A2724307A27FE
:100C9000492E080031307A2731307A2727307A27D9
:100CA0000800C000871402307E27871002307E279C
:100CB000C00012309B265A308F2612309B264614D5
:100CC0000830F50069263F08C0000830F5006926A5
:100CD0000800401C702E8426C00CF50B692E0800FD
:100CE0007526C00CF50B692E080046187E2E0000F4
:100CF00012309B2611308F260000080012308F26FC
:100D000011309B260000080046188B2E000025306D
:100D10009B264614080025308F2646100800F40054
:100D2000071002307A270000000001307A27982E41
:100D3000F40B902E0800F400071402307A2700000C
:100D4000071001307A27A42EF40B9C2E0800C00057
:100D5000BF260830F500401CB32EB926C00CF50B99
:100D6000AB2EB9260800BF26C00CF50BAB2EB9265A
:100D70000800071016307A27BD2E0000080007145F
:100D800004307A27071011307A27C62E0800A701F1
:100D9000D3012910C90B08001930C900CA0B08007B
:100DA0001930CA000608FF3A3F39A600A7000030F4
:100DB0002606031DE32EDF14D301B80AB80B03196E
:100DC0000800B803E72EDF1045132030B8002608CE
:100DD000D30029140800871329131030B900061B0B
:100DE000EE3418307A27B90BEF2E061FF52E43305C
:100DF0007A27FA2E000087170034C0010830BA00A5
:100E0000C00CC01337274518EE34C007BA0B002FAB
:100E100040080034C0010730BA0037274518EE34C7
:100E2000C007C00CC013BA0B0D2F40080034C0011E
:100E30000630BA0037274518EE34C007C00CC0137F
:100E4000BA0B1A2FC00CC01340080034C001053083
:100E5000BA0037274518EE34C007C00CC013BA0BD0
:100E6000292FC00CC013C00CC0134008003445101B
:100E70001D30B900061B432F01307A273F2FB90BD5
:100E80003A2F4514080087173630B90001307A2709
:100E9000492F061F4F2FB90B462F45140800871303
:100EA0004630B90001307A27552FB90B522F8717DA
:100EB000061F5B2F00348034061F5C2F5430B900AE
:100EC000061F682F01307A27652FB90B602F003479
:100ED000EE3408000800080008000800AF00643085
:100EE000B0002030B100B10B732FB00B712FAF0BDE
:100EF0006F2F0800FF3E031D7A2F0800AF000A3055
:100F0000B0002030B100B10B832FB00B812FAF0B9D
:100F10007F2F08008316193099002430980083121F
:100F200080309800080008000C1E942F99000800DB
:100F3000650893276608932767089327680893270F
:100F4000DB3093270800F80B0800FF30F800F90B9E
:100F50000800FF30F900FA0B08006430FA000711AE
:100F600087110712FF307E27FF307E278316031379
:100F70003F3086008312FF307E27FF307E27FF3010
:100F80007E27FF307E270B106300000083160313BB
:100F90007F308600831206080B10FF307E27071271
:0A0FA000F601F701FF307E2708007C
:1010000008000C1E012899000800473000204B30D2
:1010100000204F300020533000200D300020080009
:101020001E30A91A0730DD00A91005308A003B25C3
:1010300008308A00080029125E08D100D30AD30BB9
:1010400022282F285308C4005B084402031D2F28C0
:10105000DD0B2F28DD0A2916A91452133128A918EF
:101060001020531C3628D40AD40BD403D31C3B289D
:10107000D50AD50BD503531D4028D60AD60BD60367
:10108000D31D4528D70AD70BD703531E4A28D80AA1
:10109000D80BD803D31E4F28D90AD90BD903EE0A8F
:1010A000EE0B53285528EE0366285308C4005B084E
:1010B000C406C4050319662829160530EE00D215AA
:1010C00052121E30A91A0730DD00A9105C08C400B6
:1010D0005B08C406C405031D52165B08DE005308F6
:1010E000DE05291E8829C801C613A001A101A2019D
:1010F0007F30A300A400A500D11E83282030A000CB
:101100005908A300A628511E8A281030A0005808AC
:10111000A300AD28D11D91280830A0005708A300D6
:10112000B428511D98280430A0005608A300BB28FD
:10113000D11C9F280230A0005508A300C228511CD2
:10114000E4280130A0005408A300E428511EAD2873
:101150001030A1005808A400C928D11DB4280830B7
:10116000A1005708A400D028511DBB280430A100BD
:101170005608A400D728D11CC2280230A100550867
:10118000A400DE28511CE4280130A1005408A4006A
:10119000E428D11DD0280830A2005708A500E42873
:1011A000511DD7280430A2005608A500E428D11C00
:1011B000DE280230A2005508A500E428511CE428CE
:1011C0000130A2005408A500FF30002023087F3C16
:1011D000A300002024087F3CA400002025087F3CB9
:1011E000A50000202308003A031901292408003A29
:1011F00003190C29240823020319012903180129C2
:101200000C292508003A031934292508240203195A
:1012100051290318512934292508003A031917299F
:101220002508230203191729031851291729230810
:10123000C300EE00EE0CEE13EE01EE146E1404305B
:1012400043020318C30323082402430203182B2973
:10125000C6172108C80023082502430203186D2978
:10126000C6172208C8076D292408C300EE00EE0C3B
:10127000EE13EE01EE146E14043043020318C303A0
:1012800024082302430203184829C6172008C8006F
:1012900024082502430203186D29C6172208C8072F
:1012A0006D292508C300EE00EE0CEE13EE01EE14DE
:1012B0006E14043043020318C303250824024302BA
:1012C00003186529C6172108C80025082302430210
:1012D00003186D29C6172008C807D21A7129C6132A
:1012E0007929C61F79295108C400DA004808D100BD
:1012F0007B295108C4007F304418D400C418D5009D
:101300004419D600C419D700441AD800C41AD90009
:101310005B08DC005308DB007F30531CD400D31C77
:10132000D500531DD600D31DD700531ED800D31EA1
:10133000D9000800AF000A30B0002030B100B10B76
:101340009F29B00B9D29AF0B9B290800C40080305A
:101350000120440801200800012000300120FF3056
:10136000012008003F302806031DBD29A912323094
:101370006E27DB01DC01DE0108003F302806031D7B
:10138000C229A9122808093A0319312A28081B3A48
:101390000319392A2808083A0319412A2808193A52
:1013A0000319492A2808183A0319492A2808103A23
:1013B0000319592A2808383A0319612A2808303AAB
:1013C0000319792A2808203A0319712A2808343A7F
:1013D0000319792A2808243A0319812A2808363A59
:1013E0000319892A2808043A0319912A2808263A59
:1013F0000319992A2808063A0319992A2808023A53
:101400000319A92A2808073A0319B12A2808033A18
:101410000319C92A2808013A0319C12A28080B3AD6
:101420000319C92AA918080028083B3A0319D12A28
:1014300028081F3A0319F92A2808053A0319D12A5E
:101440002808283A0319F92A2808123A0319D12A38
:1014500028082D3A0319E32A28080C3A03190B2B04
:1014600008006D08083EA6210030AA210530AC21F5
:1014700008006D08083EA6210030AA210F30AC21DB
:1014800008006D08083EA6210330AA210330AC21D4
:1014900008006D08083EA6210A30AA210A30AC21B6
:1014A00008006D08083EA6210430AA210230AC21B4
:1014B00008006D08083EA6210530AA210030AC21A5
:1014C00008006D08083EA6210F30AA210030AC218B
:1014D00008006D08283EA6210430AA21FE30AC2168
:1014E00008006D08283EA6210330AA21FD30AC215A
:1014F00008006D08283EA6210A30AA21F630AC214A
:1015000008006D08283EA6210030AA21FB30AC213E
:1015100008006D08283EA6210030AA21F030AC2139
:1015200008006D08383EA621FD30AA21FD30AC210F
:1015300008006D08383EA621F630AA21F630AC210D
:1015400008006D08383EA621FC30AA21FE30AC21EF
:1015500008006D08183EA621FB30AA210030AC21FE
:1015600008006D08183EA621F030AA210030AC21F9
:1015700008006D08183EA621FC30AA210230AC21DB
:1015800008006D08183EA621FC30AA210430AC21C9
:1015900008006D08183EA621F630AA210A30AC21B9
:1015A00008001E306E270930A6210030AA21003025
:1015B000AC210130ED000830A6210030AA21003016
:1015C000AC21ED01B9291E306E270930A62100306B
:1015D000AA210030AC210130ED00B92932306E274C
:1015E0000C30A6210030AA210030AC210430ED00DF
:1015F000B92932306E270A30A6210030AA210030E6
:10160000AC210130ED000830A6210030AA210030C5
:10161000AC21ED01B92932306E270830A621003007
:0A162000AA210030AC21ED01B92928
:10200000820081348234843488349034A0340034A3
:102010000034003400340034C134C234003400349D
:102020000034003400340034003400340034003410
:1020300000340034003400340034C434003400343C
:1020400000340034080082000034003400340034CE
:1020500000340034003400340534003400340034DB
:1020600000340034003401340034003400340834C7
:1020700000340034003400340D34003400340034B3
:1020800000340034003400340034003400340034B0
:102090000034003400340034003400340034820052
:1020A000003411340034153400340034003400346A
:1020B0000034003400340034003400340034003480
:1020C0000034003400340034003400340034003470
:1020D0000034003400340034003400340034003460
:1020E0000034003400340034003400340034003450
:1020F00000340034003482000034003400340034F2
:102100000034003400341E340034003400342134F0
:102110000034003400340034183400340034003407
:10212000003400340034003400340034003400340F
:1021300026340034003400340034003400340034D9
:1021400000340034003400340034003400348200A1
:102150002B340034003400342E3400340034003486
:1021600000340034003400340034003400340034CF
:1021700000340034003400340034003400340034BF
:1021800000340034003400340034003400340034AF
:10219000003400340034003400340034003400349F
:1021A0000034003400348200003400340034003441
:1021B000003400340034003400340034003400347F
:1021C000393400340034003400343E3400340034F8
:1021D00000343434003400344434003400340034E7
:1021E000003400340034003400340034003400344F
:1021F00000340034003400340034003400348200F1
:10220000003448340034003400344D340034003499
:10221000003400340034003400340034003400341E
:10222000003400340034003400340034003400340E
:1022300000340034003400340034003400340034FE
:1022400000340034003400340034003400340034EE
:102250000034003400348200003400340034003490
:1022600000340034003400340034073400340034C7
:1022700000340434003400340034003400340034BA
:1022800001340034003400340034003400340034AD
:102290000F3400340034003400340034003400348F
:1022A0000034003400340034003400340034820040
:1022B0000034003415340034593400340034003410
:1022C000003400340034003400340034003400346E
:1022D000003400340034003400340034003400345E
:1022E000003400340034003400340034003400344E
:1022F000003400340034003400340034003400343E
:1023000000340034003482000034003400340034DF
:1023100000340034003400340034003400342334FA
:10232000003400340034003400341F3400340034EE
:1023300000340034003428340034003400340034D5
:1023400000343034003400340034003400340034BD
:10235000003400340034003400340034003482008F
:102360003434003400340034003438340034003461
:1023700000340034003400340034003400340034BD
:1023800000340034003400340034003400340034AD
:10239000003400340034003400340034003400349D
:1023A000003400340034003400340034003400348D
:1023B000003400340034820000340034003400342F
:1023C000003400340034003400344234003400342B
:1023D00000340034003400340034003400343E341F
:1023E000003400340034003400344B3400344734BB
:1023F000003400340034003400340034003400343D
:1024000000340034003400340034003400348200DE
:10241000003400344E34533400340034003400347B
:10242000003400340034003400340034003400340C
:1024300000340034003400340034003400340034FC
:1024400000340034003400340034003400340034EC
:1024500000340034003400340034003400340034DC
:10246000003400340034820000340034003400347E
:1024700000340034003408340034003400340034B4
:1024800000340034003401340034003400340034AB
:102490000034003400340D3400340034003414347B
:1024A000003400340034003400340034003400348C
:1024B000003400340034003400340034003482002E
:1024C0001734003400341A3400340034003400343B
:1024D000003400340034003400340034003400345C
:1024E000003400340034003400340034003400344C
:1024F000003400340034003400340034003400343C
:10250000003400340034003400340034003400342B
:1025100000340034003482000034003400340034CD
:10252000003400340034003400340034003400340B
:1025300000342734003400340034003400340034D4
:102540000034213400340034003431340034003499
:1025500000342B34003400340034003400340034B0
:10256000003400340034003400340034003482007D
:10257000003400343634003400343D340034003448
:1025800000340034003400340034003400340034AB
:10259000003400340034003400340034003400349B
:1025A000003400340034003400340034003400348B
:1025B000003400340034003400340034003400347B
:1025C000003400340034820000340034003400341D
:1025D00000340034003400344A3400340034003411
:1025E00051340034003400344134003400340034B9
:1025F0004E340034003400340034003400340034ED
:10260000003400340034003400340034003400342A
:1026100000340034003400340034003400348200CC
:10262000003454340034003457340034003400345F
:1026300000340034003400340034003400340034FA
:1026400000340034003400340034003400340034EA
:1026500000340034003400340034003400340034DA
:1026600000340034003400340034003400340034CA
:06267000003400340034C8
:103000008200013402340F3403341B3413342E3461
:1030100004342A342434103421341C3414342F342E
:10302000053423343B34113420341D34153430340A
:103030000734083409342C340A342934263438341B
:10304000063422341F3412342B341E3416343134F7
:103050001734183419343A341A343C3428343E3492
:103060000B340C340D3425340E3427342D343F34D6
:1030700032343334343436343534373439343D34FF
:103080000034003482001534133410343B343834A7
:103090000034003479340034003400340034003417
:1030A0000034003400340034003400340034003480
:1030B0000034003400340034003400340034003470
:1030C000003400341634543457340034003400349F
:1030D000003400340034003400341C340034003434
:1030E0000034003400340034003402340734043433
:1030F0000D340E340B34083419341A3401341F34AF
:063100000034003400342D
:1032000082000134023403340434053406340734B4
:10321000083409340A340B340C340D340E340F34B2
:103220001034113412341334143415341634173462
:10323000183419341A341B341C341D341E341F3412
:1032400020342134223423342434253426342734C2
:10325000283429342A342B342C342D342E342F3472
:103260003034313432343334343435343634373422
:10327000383439343A343B343C343D343E343F34D2
:103280004034413442344334443445344634473482
:10329000483449344A344B344C344D344E344F3432
:1032A00050345134523453345434553456345734E2
:1032B000583459345A345B345C345D341F34203410
:1032C000213422342334243425342634273428343A
:1032D00029342A342B342C342D342E342F343034EA
:1032E000313432343334343435343634373438349A
:1032F00039343A343B343C343D343E343F3440344A
:1033000041344234433444344534463447344834F9
:1033100049344A344B344C344D344E344F345034A9
:103320005134523453345434553456345734583459
:1033300059345A345B345C345D345E345F34603409
:1033400061346234633464346534663467346834B9
:103350002A342B342C342D342E342F343034313461
:103360003234333434343534363437343834393411
:103370003A343B343C343D343E343F34013402343F
:1033800003340434053406340734083409340A3469
:103390000B340C340D340E340F3410341134123419
:1033A00013341434153416341734183419341A34C9
:0833B0001B341C341D341E34D3
:103400008200613462346334643465346634673412
:10341000683469346A346B346C346D346E346F34B0
:103420007034713472347334743475347634773460
:10343000783479347A347534613461346F342E34AD
:103440002C3421343F342D3427345C342F34203451
:103450007E345E34FF341D34163415342B342B3453
:103460002B342B344C342C342C342C343C34183442
:10347000FF340F34FF34FF34FF34FF34FF34FF34A4
:103480003134323433343434353436343034373400
:10349000383439340A34203426340A342B34253471
:1034A000203420342A34203424342034283428345E
:1034B0003C342934293429343E3429343A343B34D9
:1034C00020342034203422342A342A342034203446
:1034D00020342034FF34FF34FF34FF34FF34FF3412
:1034E000FF34FF34FF34FF34FF34FF34FF34FF3444
:1034F000FF34FF34FF34FF34FF34FF34FF34FF3434
:10350000FF348200FF342034FF34FF342134FF3491
:10351000FF341E34FF34FF340A3419341F340A34A4
:1035200029342934FF342D3419343C34FF34FF342A
:103530002C34FF341834FF342B34FF34FF34FF3481
:10354000FF34FF34FF34FF34FF34FF34FF34FF34E3
:10355000FF34FF34FF34FF341D341634153428345F
:10356000203420342B342A34213421342C343B347D
:10357000183428340F34FF34FF34FF34FF34FF3461
:10358000FF34003401340234033404340534093484
:103590000634073408340A34FF34FF34FF34FF3470
:1035A000FF34FF34FF34FF34FF34FF34FF34FF3483
:1035B000FF34FF34FF34FF34FF34FF34FF34FF3473
:1035C000FF34FF34FF34FF34FF34FF34FF34FF3463
:1035D000FF34FF34FF34FF34FF34FF34FF34FF3453
:1035E000FF34FF34FF34FF34FF34FF34FF34FF3443
:1035F000FF34FF34FF34FF34FF34FF34FF34FF3433
:103600008200043424340534023423340334FF3478
:10361000FF34FF34FF340A3419341F340A34293498
:103620002934FF342D3419343C34FF34FF342C3426
:10363000FF341834FF342B34FF34FF34FF34FF34AD
:10364000FF34FF34FF34FF34FF34FF34FF34FF34E2
:10365000FF34FF34FF341D34163401342834203451
:1036600020342B342A34213421342C343B34183484
:1036700028340F34FF34FF34FF34FF34FF34FF3479
:10368000003401340234033404340534093406347C
:10369000073408340A34FF34FF34FF34FF34FF3476
:1036A000FF34FF34FF34FF34FF34FF34FF34FF3482
:1036B000FF34FF34FF34FF34FF34FF34FF34FF3472
:1036C000FF34FF34FF34FF34FF34FF34FF34FF3462
:1036D000FF34FF34FF34FF34FF34FF34FF34FF3452
:1036E000FF34FF34FF34FF34FF34FF34FF34FF3442
:1036F000FF34FF34FF34FF34FF34FF34FF34FF3432
:103800008200103415341434003409341334003475
:103810001434083401341434003419340F3415349A
:103820000034023415341434003404340F340034BA
:103830001134153409341434053400340834053493
:1038400000340C3409340B34053400341434083497
:1038500005341934003401340D3400340534013496
:103860000334083400340034163405341234193467
:1038700000340D3415340334083400341234093460
:103880000734083414340034193405341334003444
:103890000234053405340E340034063412340F3447
:1038A0000D3400340034003400340034003400346B
:1038B0000034003400340034003400340034003468
:1038C0000034003400340034003400340034003458
:1038D0000034003400340034003400340034003448
:1038E0000034003400340034003400340034003438
:0E38F00000340034003400340034003400345E
:103A000082001534103400340E340F340034033483
:103A1000053412341434013409340E3400341434AF
:103A20000834053412340534003403340F340D34B3
:103A300005340034003400340034003400340134E0
:103A40001234053400340C340F340E34073400348F
:103A50000534183401340D3410340C34053400347A
:103A60000F3406340634003401340C340C34003482
:103A700006340934123413341434003414340F343B
:103A80000F3400340A341534133414340034013440
:103A90000E3419340034173405340034033401343F
:103AA0000D340534003404340F340E34243414340B
:103AB000003405341634053412341934003400341B
:103AC0000034003400340034003400340034003456
:103AD0000034003400340034003400340034003446
:103AE0000034003400340034003400340034003436
:103AF0000034003400340034003400340034003426
:103C00008200103405340F3410340C340534003481
:103C100008340134163405340034053418340334C0
:103C2000153413340534003401340E3400340134B7
:103C30001434003404341534123409340E34073487
:103C400000341634093413340934143400340E3477
:103C50000F34143400340F340634143405340E3465
:103C600000341734083405340E3400340334083477
:103C700001340E3407340534003406340F34123462
:103C800000341134153405341334143409340F342A
:103C90000E3400343B34093400340034153413340A
:103CA00000340D3405340034023405340034053456
:103CB000163405340E34003400340034003400343B
:103CC0000034003400340034003400340034003454
:103CD0000034003400340034003400340034003444
:103CE0000034003400340034003400340034003434
:103CF0000034003400340034003400340034003424
:02400E00313F40
:00000001FF
